:1000000017C039C038C037C036C035C034C033C05F
:1000100032C031C030C02FC02EC02DC02CC0031440
:100020006EE6FFFFFFFF000000000007385A89FF5F
:1000300011241FBECFE5D1E0DEBFCDBF20E0A0E69A
:10004000B0E001C01D92A138B207E1F7E1E6F0E0AF
:10005000128281E08683ABE6B0E09EEF15969C931A
:1000600015979DEF17969C93808788E58187612C73
:10007000712C71D0A5C0C4CF20ED37E0019720F0DE
:10008000F9013197F1F7FACF089588EE93E0F4CFB4
:1000900081EA87B986EC86B9369A0895369A3699F8
:1000A000FECF85B10895CF92DF92EF92FF920F932A
:1000B0001F93CF93C82F8B018FE1E82E80E0F82E9D
:1000C00098E2C92E90E0D92ECC2381F0F7018491DB
:1000D00089BDF601849188BDC801CEDF19BC18BC6A
:1000E000C801CADFC801C8DFC150EECFCF911F9150
:1000F0000F91FF90EF90DF90CF900895CF93DF9313
:10010000D82F64E170E08AE0CEDF84EF91E0B4DFC5
:100110008D2F64E649D0CAE06C2F46D0892F68EC59
:1001200070E0C1DFB2DF8D2F6C2F3ED0D92F3CD0D5
:10013000892F68EC70E0B7DFA8DF68EC70E08D2FE6
:10014000B2DFA3DF64E170E08AE0ADDF84EF91E02D
:10015000DF91CF9191CF83EA87B986EC86B9369942
:10016000FECF369A3699FECF85B18FE384BBBB9A1A
:10017000C39AB99AB89A81E08ABD83BF8AB5806272
:100180008ABD8AB580688ABD97B328B3892F90E06D
:10019000809590958B7F822B88BB7ADF8CE291E0F3
:1001A0006BDF7CDFABDFFACF991B79E004C0991FCE
:1001B000961708F0961B881F7A95C9F780950895C1
:0401C000F894FFCFE1
:00000001FF
